:03000000020008F3
:0300610002000397
:0500030012006480FE04
:100064009090007407F0909002E4F0909003F0E414
:10007400909004E0FA20E1F8909014E0FA90901047
:03008400F080ED1C
:06003700E478FFF6D8FD9D
:100015007900E94400601B7A0090008B780075A098
:1000250000E493F2A308B8000205A0D9F4DAF2754A
:02003500A0FF2A
:10003D007800E84400600A790075A000E4F309D85F
:10004D00FC7800E84400600C7900900000E4F0A317
:04005D00D8FCD9FAF8
:0D00080075810C120087E582600302000381
:04008700758200225C
:00000001FF
